:020000040000FA
:020000000528D1
:0800080014288316FF30850067
:1000100000308600831286019301640005181520C4
:100020001308940086000D280D2893015520051C07
:1000300054285520051C54285520051C54285520AB
:10004000051C542805182228051C242855200518AD
:1000500013145520051C2A285520051893145520E3
:10006000051C30285520051813155520051C362869
:100070005520051893155520051C3C2855200518BA
:1000800013165520051C4228552005189316552097
:10009000051C48285520051813175520051C4E2807
:1000A000552005189317552008001430910014307E
:0E00B0009000900B5928910B5728640008000F
:00000001FF
